:40000000FFFF011EFFFFFFFFFFFFFFFF0E37FFFFFFFFFFFFFFFFFFFFFFFFFFFFFFFFFFFFFFFFFFFFFFFFFFFFFFFFFFFFFFFFFFFFFFFFFFFFFFFFFFFFFFFFFFFFFFFFAF5097
:40004000E450E51FE8EEEFFE50EE50EF50E670E570E470E629100102D8FFD0AFE8102FFD09100102B0E5B0E450E650E770EF70EE1FE8FFEEEE2F28EE5FFF38EE4FFEC4E60C
:4000800070E570E4E4E3E470E2E4E1E2F4E2E4E0E5F4E4022550E4E4E1E5F4E4022550E450E5AF70E4E4E0E4B24256E4804200DB0960E060E1A0E046E4084222DB0660E2F6
:4000C00060E3A0E2D600DE4244DB0660E160E0A0E0F0E4DB0660E360E2A0E250E4AF70E970EA70EB9C10B0EBB0EA021110E010EB10EA7B07A2B31FA2A27B0522B332A21E18
:400100009AE8E4EBE3E4EAE250EB50EA50E9AF50E650E71FE8EEEFFE50EE50EFC4E601E0E9000FFFE9040FFE0C002C00A6E2006B05B1E00E2AFB2C013C000C001C05E4E0E8
:40014000E442416B0BB0E496E4E2A0E280E0EBF70C001C003C004C0042336B04C3403AFC0C011C052C0E3CDE4C005C08E4E4E642656B0DC26296E6E0A0E0A0E280E4EBF35E
:40018000E9000102D6003EB2FFB2EED60BD8D6003E8BFE5C02D6006689E8FE89E9FFB0ECDCFFB0EABC08B0E8B0E9D60CC5B0ECDCFFB0EABC08B0E89C09D60CC5B0ECDC023E
:4001C000B0EABC37B0E89C01D60DBDB0ECDC02ACFFBCC9B0E89C05D60DBDB0ECDC02B0EABC37B0E89C0BD60DBDB0ECDC0288AEFE88BEFFB0E89C02D60DBDB0E89C06D60E4D
:40020000B44200ED03DCB0ECDC02882EFE883EFF60E260E3A0E21FE8EE2EEAB0E89C06D60DBDB0ECDC02B0EAB0EBB0E89C01D60DBDB0E89C06D60EB44200ED03DCB0ECDC3F
:400240000288AEFE88BEFFB0E89C0CD60DBDB0ECDC02B0EAB0EBB0E89C05D60DBDB0E89C06D60EB44200ED03DCB0ECDC02B0EAB0EBB0E89C0BD60DBDB0E89C06D60EB44219
:4002800000ED03DCB0ECDC03882EFE883EFF60E260E3A0E21FE8EE2EEAB0E89C02D60DBDB0ECDC0388AEFE88BEFFB0E89C06D60DBDB0ECDC03882EFE883EFF60E260E3A0AD
:4002C000E21FE8EE2EEAB0E89C0CD60DBDB0ECDC02B0EABC37B0E89C03D60DBDB0ECDC02ACFFBCC9B0E89C07D60DBDB0ECDC02ACFFBCC9B0E89C0DD60DBDB0ECDC02882E11
:40030000FE883EFF60E260E3A0E21FE8EE2EEAB0E89C08D60DBDB0E89C06D60EB44200ED03DCB0ECDC0288AEFE88BEFFB0E89C04D60DBDB0ECDC02B0EAB0EBB0E89C07D69F
:400340000DBDB0E89C06D60EB44200ED03DCB0ECDC02882EFE883EFF60E260E3A0E21FE8EE2EEAB0E89C0ED60DBDB0ECDC02B0EAB0EBB0E89C03D60DBDB0E89C06D60EB492
:400380004200EB58B0ECDC02B0EAB0EBB0E89C0DD60DBDB0E89C06D60EB44200EB3EB0ECDC04880EFE881EFF60E060E1A0E01FE8EE0EEAB0E89C04D60DBDB0ECDC0488AEBE
:4003C000FE88BEFFB0E89C08D60DBDB0ECDC0488AEFE88BEFFB0E89C0ED60DBDD6010FAFD600648CFF9CDDD60193D6010FAFD60064B0E89C23D60193D6010FAFD60064B0BB
:40040000ECDCFFB0EABC08B0E8B0E9D60CC5B0ECDCFFB0EABC08B0E89C09D60CC5B0ECDC03B0EAB0EBB0E89C01D60DBDB0ECDC03B0EAB0EBB0E89C03D60DBDB0ECDC03B0CF
:40044000EAB0EBB0E89C0BD60DBDB0ECDC03B0EAB0EBB0E89C07D60DBDB0ECDC03B0EAB0EBB0E89C05D60DBDB0ECDC03B0EAB0EBB0E89C0DD60DBDB0E89C06D60EB442005F
:40048000ED05F5B0ECDC02B0EABC37B0E89C01D60DBDB0ECDC02ACFFBCC9B0E89C05D60DBDB0ECDC02B0EABC37B0E89C0BD60DBDB0E89C06D60EB44200ED05F5B0ECDC029B
:4004C000B0EABC1EB0E89C02D60DBDB0ECDC02B0EAB0EBB0E89C06D60DBDB0ECDC02ACFFBCE2B0E89C0CD60DBDB0E89C06D60EB44200ED05F5B0ECDC02B0EAB0EBB0E89CA8
:4005000001D60DBDB0ECDC02B0EAB0EBB0E89C05D60DBDB0ECDC02B0EAB0EBB0E89C0BD60DBDB0E89C06D60EB44200ED05F5B0ECDC02B0EABC37B0E89C03D60DBDB0ECDCB3
:4005400002ACFFBCC9B0E89C07D60DBDB0ECDC02ACFFBCC9B0E89C0DD60DBDB0E89C06D60EB44200ED05F5B0ECDC02B0EAB0EBB0E89C04D60DBDB0ECDC02ACFFBCE2B0E806
:400580009C08D60DBDB0ECDC02B0EABC1EB0E89C0ED60DBDB0E89C06D60EB44200EB56B0ECDC02B0EAB0EBB0E89C03D60DBDB0ECDC02B0EAB0EBB0E89C07D60DBDB0ECDC4A
:4005C00002B0EAB0EBB0E89C0DD60DBDB0E89C1ED60EB4B0ECB0EDB0EABC08B0E8B0E9D60CC5B0ECB0EDB0EABC08B0E89C09D60CC5E900010CD6010FAF5C02D6006689E879
:40060000FE89E9FFB0ECDCFFB0EABC08B0E8B0E9D60CC5B0ECDCFFB0EABC08B0E89C09D60CC5B0ECDC02B0EABC2DB0E89C01D60DBDB0ECDC02ACFFBCD3B0E89C05D60DBD86
:40064000B0ECDC02B0EABC2DB0E89C0BD60DBDB0E89C05D60EB44200ED07E4B0ECDC0288AEFE88BEFFB0E89C02D60DBDB0ECDC0288AEFE88BEFFB0E89C06D60DBDB0ECDCA5
:400680000288AEFE88BEFFB0E89C0CD60DBDB0E89C08D60EB44200ED07E4B0ECDC02B0EAB0EBB0E89C01D60DBDB0ECDC02B0EAB0EBB0E89C05D60DBDB0ECDC02B0EAB0EB36
:4006C000B0E89C0BD60DBDB0E89C05D60EB44200ED07E4B0ECDC02B0EABC2DB0E89C03D60DBDB0ECDC02ACFFBCD3B0E89C07D60DBDB0ECDC02ACFFBCD3B0E89C0DD60DBD38
:40070000B0E89C05D60EB44200ED07E4B0ECDC0288AEFE88BEFFB0E89C04D60DBDB0ECDC0288AEFE88BEFFB0E89C08D60DBDB0ECDC0288AEFE88BEFFB0E89C0ED60DBDB0AF
:40074000E89C08D60EB44200ED07E4B0ECDC02B0EAB0EBB0E89C03D60DBDB0ECDC02B0EAB0EBB0E89C07D60DBDB0ECDC02B0EAB0EBB0E89C0DD60DBDB0E89C05D60EB44288
:4007800000EB61B0ECDC03B0EAB0EBB0E89C02D60DBDB0ECDC03B0EAB0EBB0E89C04D60DBDB0ECDC03B0EAB0EBB0E89C0CD60DBDB0ECDC03B0EAB0EBB0E89C08D60DBDB013
:4007C000ECDC03B0EAB0EBB0E89C06D60DBDB0ECDC03B0EAB0EBB0E89C0ED60DBDB0E89C08D60EB4D6010FAFD600648CFF9CBAD605F9D6010FAFD60064B0E89C46D605F918
:40080000D6010FAFD60064B0ECDCFFB0EABC08B0E8B0E9D60CC5B0ECDCFFB0EABC08B0E89C09D60CC5B0ECDC02B0EABC2DB0E89C0BD60DBDB0ECDC02B0EABC50B0E89C0C47
:40084000D60DBDB0E89C05D60EB44200ED0AFFB0ECDC01B0EAB0EBB0E89C0BD60DBDB0E89C05D60EB44200ED0AFFB0ECDC02ACFFBCD3B0E89C0DD60DBDB0ECDC02ACFFBCC3
:40088000B0B0E89C0ED60DBDB0E89C05D60EB44200ED0AFFB0ECDC01B0EAB0EBB0E89C0DD60DBDB0E89C05D60EB44200ED0AFFB0ECDC02B0EABC2DB0E89C03D60DBDB0EC95
:4008C000DC02B0EABC50B0E89C04D60DBDB0E89C05D60EB44200ED0AFFB0ECDC01B0EAB0EBB0E89C03D60DBDB0E89C05D60EB44200ED0AFFB0ECDC02ACFFBCD3B0E89C0518
:40090000D60DBDB0ECDC02ACFFBCB0B0E89C06D60DBDB0E89C05D60EB44200ED0AFFB0ECDC01B0EAB0EBB0E89C05D60DBDB0E89C0AD60EB44200ED0AFFB0ECDC05B0EABC3B
:400940003CB0E89C0BD60DBDB0ECDC05ACFFBCC4B0E89C0DD60DBDB0E89C0AD60EB4B0ECDC02B0EABC50B0E89C02D60DBDB0ECDC02ACFFBCB0B0E89C08D60DBDB0E89C0561
:40098000D60EB44200ED0AFFB0ECDC02B0EABC2DB0E89C01D60DBDB0ECDC02ACFFBCD3B0E89C07D60DBDB0E89C05D60EB44200ED0AFFB0ECDC02B0EAB0EBB0E89C01D60D36
:4009C000BDB0ECDC02B0EAB0EBB0E89C07D60DBDB0E89C05D60EB44200ED0AFFB0ECDC02B0EABC2DB0E89C01D60DBDB0ECDC02ACFFBCD3B0E89C07D60DBDB0E89C05D60E29
:400A0000B44200ED0AFFB0ECDC02B0EAB0EBB0E89C01D60DBDB0ECDC02B0EAB0EBB0E89C07D60DBDB0E89C05D60EB44200ED0AFFB0ECDC02B0EAB0EBB0E89C02D60DBDB07E
:400A4000ECDC02B0EAB0EBB0E89C08D60DBDB0E89C05D60EB44200ED0AFFB0ECDC02B0EABC2DB0E89C01D60DBDB0ECDC02ACFFBCD3B0E89C07D60DBDB0E89C05D60EB4421E
:400A800000EB7CB0ECDC02B0EAB0EBB0E89C01D60DBDB0ECDC02B0EAB0EBB0E89C07D60DBDB0E89C05D60EB44200EB53B0ECDC02B0EABC2DB0E89C01D60DBDB0ECDC02AC78
:400AC000FFBCD3B0E89C07D60DBDB0E89C05D60EB44200EB2AB0ECDC02B0EAB0EBB0E89C01D60DBDB0ECDC02B0EAB0EBB0E89C07D60DBDB0E89C05D60EB442006D095ED69A
:400B0000010FAFD60064B0ECDCFFB0EABC08B0E8B0E9D60CC5B0ECDCFFB0EABC08B0E89C09D60CC5B0ECDC02B0EABC2DB0E89C01D60DBDB0ECDC02B0EABC50B0E89C02D658
:400B40000DBDB0E89C05D60EB44200ED0BD4B0ECDC01B0EAB0EBB0E89C01D60DBDB0E89C05D60EB44200EB6CB0ECDC02ACFFBCD3B0E89C07D60DBDB0ECDC02ACFFBCB0B00F
:400B8000E89C08D60DBDB0E89C05D60EB44200EB43B0ECDC01B0EAB0EBB0E89C07D60DBDB0E89C05D60EB44200EB29B0ECDC05B0EAB0EBB0E89C0BD60DBDB0ECDC05B0EA70
:400BC000B0EBB0E89C0DD60DBDB0E89C14D60EB4E900010CD6010FAFD60064D60C6B8FD60E919FB0E89C0AD60EB4D603FCA9000106EB2C840FD31FC0E0E4E0E1940FD3A989
:400C0000000FD3EB04E9800FD3840FDB0200940FDBA9000FDBEB04E9010FDBE9040106A920010CEB03D60B03A9C0010CEB03D60804A980010CEB03D603E0A940010CEB03B1
:400C4000D603EEA960010CEB03D607F6A9A0010CEB03D607E8A990010CEB03D603FCB0E89C01D60EB48B86D6010FAFD60064E9010FD0E9000FD1E9010FD4E9100FD5E901F1
:400C80000FD8E9F00FD9E9020FDCE9000FDDE9010FDCE9000FDDE9030FDCE9000FDDE9FF0FD7E9010FDFD6010FAFD6006459DF0FD769100FD66BFA49200FD779100FD66B0D
:400CC000FAD6010FAF5C05D60066A6E9091FA6E8009B0459FE0FD7A6E9091FA6E8001B13A6E9111FA6E8009B0A59FD0FD706E9F816E8FFA6E9111FA6E8001B13A6E9191FE0
:400D0000A6E8009B0A59FB0FD706E9F016E8FFA6E9191FA6E8001B0A59F70FD706E9E816E8FFE4E9E256E20FF0E256E2F0422B8B0BA6E1091FA6E0001B088B49B0E01C011A
:400D40008BEF66ED01EB0649010FDF8B0459FE0FDFD0ECC0ED89EDFF89ECFE89E0FD89E1FC89E2FBD60CAA882EFB881EFC880EFD88CEFE88DEFFA0E08BB7A6E1091FA6E003
:400D8000001B088B30B0E01C018BEF66E201EB0649010FDF8B0459FE0FDFD0E289E0FD89E1FC89E2FBD60CAA882EFB881EFC880EFDA0E08BC5490F0FD7D6010FAF5C06D6B7
:400DC000006689E8FE89E9FF89EAFC89EBFD89ECFA89EDFB881EFA880EFB06E08016E10089E1FA89E0FBB0E23C64880EFC881EFDD600801FE8EE2EE0B0E23C5AD600A3B086
:400E0000E32C960221123089E3FC89E2FD88CEFC88DEFDB0EABC02888EFE889EFFD60CC588CEFA88DEFBB0EABC01888EFE889EFFD60CC5D6010FAFC8FFD0D6005CE8FDA11F
:400E40000B59F0010B09FF0105A9000105EB3EE90A0105A90001062B0409FF0106A90001072B0409FF0107A90001082B0409FF0108A90001092B0409FF0109A900010A2B90
:400E80000409FF010A0901010419000103D6003FBFD60064E9060F00E9C00F01E9060F02E9C00F03E9E90F0749200FC159DF0FC2D6010FAFD60064949106A90001062B1858
:260EC000A810C10B6BF4A900010B3BEEE9000106E810B10C0C018B02B0E0D6010FAF0A00000000000000DD
:00000001FF
